:100000000C94D5000C94F2000C94F2000C94F200C5
:100010000C94C1040C94F2000C94F2000C94F200C5
:100020000C94F2000C94F2000C9401010C94020167
:100030000C94F2000C94F2000C94F2000C94F20078
:100040000C94F2000C94F2000C94F2000C94F20068
:100050000C94F2000C94F2000C94F2000C94F20058
:100060000C94F2000C94F2000C94F2000C94F20048
:100070000C94F2000C94F2000C94F2000C94F20038
:100080000C9470040C94F2000C94F2000C94F200A6
:100090000C94F2000C94F2000C94F2000C94F20018
:1000A0000C94F2000C94F2000C94F2001201000285
:1000B00000000040EB03452000010102030109029A
:1000C0002000010100801909040000020806500008
:1000D00007058102400000070502024000000403FA
:1000E00007042C03540055002000430068006500FD
:1000F0006D006E00690074007A002C00200045003D
:100100006E00610073002B005A0066004D002C0346
:100110003500BC0022002D004400690073006B0014
:1001200065007400740065006E006C00610075006D
:1001300066007700650072006B00300368006500A0
:10014000680061004000680072007A002E007400B0
:1001500075002D006300680065006D006E00690089
:1001600074007A002E00640065000000537472650C
:10017000616D6572205149432D38300038222D4C75
:100180006175667765726B0035BC222D4C617566B2
:100190007765726B0033BD222D4C61756677657291
:1001A0006B004368616F7343680011241FBECFEF7B
:1001B000DAE0DEBFCDBF11E0A0E0B1E0ECE1F1E1BB
:1001C00002C005900D92A036B107D9F713E0A0E662
:1001D000B1E001C01D92A139B107E1F70E9403010E
:1001E0000C948C080C9400001092710014B815B88F
:1001F00017B818B81AB81BB81DB81EB810BA11BA7B
:10020000089518951895FF920F931F9381E080939E
:10021000E0008DEE8093640089E18093650080E8C2
:1002200080BF81E18093D8000E94D502789412E0CB
:1002300084E0F82E08E08091E10080FD02C081E0BA
:1002400001C085E083BF8091E10080FD02C089E0AC
:1002500001C088E1F8948093E2001093E900F092E5
:10026000F0001092E9000093F00078948895F894DB
:100270001092F0001093E9001092F0007894109220
:10028000E2000E94D502D7CF2FEF25B98BE484B9C5
:1002900080EC88B990E497B92BB987EA8AB99EB9FE
:1002A0009DB983EF81BB80EF80BB0E943B03089523
:1002B000482F81E08093E9008091E80080FF02C030
:1002C00080E0089580EA8093E800242F392FC90147
:1002D000FC0103C081918093F1008091E80085FDCD
:1002E000F9CF1092E80081E00895482F82E08093D2
:1002F000E9008091E80082FD02C080E0089580EA74
:100300008093E800242F392FC901FC0103C080919C
:10031000F10081938091E80085FDF9CF1092E8000B
:1003200081E00895FC0140916001509161019B01C1
:10033000461757070CF49A014EEF9091E800892F69
:100340008570D9F392FD18C02134310514F080E492
:1003500001C0822F182E26FC059026FE01900092E7
:10036000F1001A94C1F7281B31094093E8002115C8
:10037000310519F7803409F30895CB0108951092DF
:10038000E9009091E80093FF0FC15091F100609156
:10039000F1007091F100F091F100E091F100809195
:1003A000F1008091F1004091F100937F9093E8007B
:1003B000342F20E090E0282B392B309361012093DB
:1003C0006001513209F483C0523248F4513009F4CB
:1003D00053C05130A0F0523009F0E3C051C0513841
:1003E00009F4B3C0523820F4503809F0DAC073C0B1
:1003F000523809F4B3C0513A09F0D3C0C6C06330D3
:1004000061F0643020F4613009F0CBC006C0653083
:1004100041F0693009F0C5C00FC0713009F0C1C0AA
:10042000BCC08EEF8093E8008091E8008570E1F316
:1004300070687093E3000895723008F0B2C08EEFD8
:100440008093E800272E7723A9F091E09093E900AC
:100450009093EB0081E88093EC0026E32093ED007D
:1004600082E08093E9009093EB0080E88093EC00B9
:100470002093ED008EE726C06B3009F092C08DC04E
:10048000613019F0633009F08CC0772309F089C01E
:100490002E2F2F77233008F084C08EEF8093E80052
:1004A0002093E90061FF04C081E28093EB0008958E
:1004B00089E18093EB0081E090E002C0880F991FF2
:1004C0002A95E2F78093EA001092EA0008956F3FC0
:1004D00009F067C062C0663061F0683069F1662378
:1004E00009F05FC08091E8008570E1F31092F1009F
:1004F00052C080E4282AF23031F0F33059F0F13064
:1005000009F04FC004C060E2EEEBF0E010C0ECEA8E
:10051000F0E00CC0743008F044C0EEEDF0E077235A
:1005200029F08491E80FF11D7150F9CF6491CF014A
:1005300070E00E94920108958091E8008570E1F3D7
:10054000822D81708093F10028C06A3051F5E2302D
:1005500040F58091E8008570E1F31DC0662309F540
:100560008091E8008570E1F3E770E093E900809105
:10057000EB0090E025E0969587952A95E1F781704C
:100580001092E9008093F10006C06E3F51F4809113
:10059000E8008570E1F31092F1008EEF8093E8009F
:1005A000089581E28093EB0008951F938091DA0013
:1005B00080FD08C08091D90080FF25C08091E000B7
:1005C000882309F11092DA008091D90080FF11C0D0
:1005D00081E08093D70081EB8093D80082E189BDD0
:1005E00009B400FEFDCF81E98093D8001092E000AD
:1005F00007C081E18093D80080E189BD1092D700C7
:100600001092E10022248091E10091E09093E100BA
:10061000182F83FF0DC01092E9001092EC0082E3C6
:100620008093ED009093EB0084E08093E800222417
:1006300010FF0BC08091D80085FD07C080EB809330
:10064000D80080E189BD0E94F40014FF0EC08091A3
:10065000D80085FF0AC082E189BD0E94440109B427
:1006600000FEFDCF80E98093D8000E94BF010E9468
:1006700082051F910895E0E0F1E02FEF96E089E216
:1006800004C02583908B818B739631E0E331F307AF
:10069000C0F32F010895CF93DF93DC0175E0FC01D7
:1006A00071936EE111966C93DF011196E2012A8538
:1006B0003B85832F992787FD9A958183FD0131968C
:1006C00011962C93DF0111968D858183ED01219682
:1006D000F201848511968C93DE0111962085318577
:1006E000832F992787FD9A958983FD01319611966D
:1006F0002C931182D2011E968C911E9782837E8745
:100700006F87FE0177968C9180FD03C02CE231E06B
:1007100002C028E631E081E08F8B21839F012C5FAE
:100720003F4FC901DF91CF9108955F9AF201238174
:100730002B5F40E25EE40DC0215019F426E032E860
:100740000FC01B9ACA010197F1F71B9ACA010197C2
:10075000F1F71A99F1CF158284E1868320E030E029
:10076000C90108951F93182FF201858187FF05C0E5
:100770000E9495039C01009711F5F2018581912F4C
:10078000981B892F81F097FD02C05F9802C05F9A85
:100790008195282F220F40E85EE31B9ACA0101973A
:1007A000F1F72150D1F717FD0DC0112361F01A9B0D
:1007B0000AC081E0828B8FEF858322E033E8C90194
:1007C0001F91089510E0158384E1868320E030E0D6
:1007D000F6CFD20117968C911797813061F0813056
:1007E00028F0823069F08330A9F40FC08D9A469AC0
:1007F0005A9A8E9818C08E9A469A5A9A8D9815C011
:100800008E9A8D9A5A9A469812C08E9A8D9A469AC6
:100810005A980FC0813049F0813028F0823039F089
:10082000833041F406C08C9805C08F9803C0299886
:1008300001C0599881E1809365008BE0809391001D
:1008400087EA91E6909399008093980082E08093E4
:10085000710080ED97E00197F1F716968C9116974D
:10086000882399F414961C92149780E88093690069
:1008700088E08CBB8DBB80ED97E020E931E0F90189
:100880003197F1F70197D9F71DBA84E116968C9349
:10089000169714968C91882319F020E030E00DC053
:1008A0008FEF0E94B2031D9B03C02AE332E805C00C
:1008B00081E0F201848328E236E8C901089581309D
:1008C00049F0813028F0823039F0833041F406C09D
:1008D0008E9A08958D9A0895469A08955A9A089581
:1008E0001F920F920FB60F9211241F932F933F93D5
:1008F0004F935F936F937F938F939F93AF93BF9328
:10090000CF93DF93EF93FF93C0E0D1E010E08E81AF
:100910008823C9F081508E83882311F01F5F13C094
:100920008F81813049F0813028F0823039F0833076
:1009300041F406C08C9A05C08F9A03C0299A01C061
:10094000599A0E945F04639681E0CC34D807F9F687
:10095000112319F489E180936500FF91EF91DF91F4
:10096000CF91BF91AF919F918F917F916F915F9147
:100970004F913F912F911F910F900FBE0F901F909D
:1009800018951F920F920FB60F9211248F93EF9329
:10099000FF9381E0F2018483FF91EF918F910F909B
:1009A0000FBE0F901F901895AC0121C061347105E6
:1009B00014F090E401C0962F8091E80080FFFCCFF6
:1009C0008091E8008E7F8093E800292FFA018191C1
:1009D0008093F1002150D9F78091E8008F778093C0
:1009E000E800892F90E0480F591F681B790B6115AB
:1009F0007105E1F60895AC0121C06134710514F070
:100A000090E401C0962F8091E80082FFFCCF809196
:100A1000E8008B7F8093E800292FFA018091F10094
:100A200081932150D9F78091E8008F778093E80077
:100A3000892F90E0480F591F681B790B61157105CC
:100A4000E1F608958091720190E083709070892B97
:100A500009F04DC080917301882309F048C0F2016C
:100A6000E081EE2319F0E03531F402C08FE101C0DE
:100A700081E08093820180E88093830181E080930C
:100A800085018FE1809386018AE891E062EA71E056
:100A90000E947E08F201808190E08E7F9070843009
:100AA000910569F0853091051CF4029789F423C003
:100AB0008830910539F08035910551F406C068E819
:100AC00071E01BC06CE771E018C06CE671E015C006
:100AD00080E38093A20188E38093A30181E3809364
:100AE000A40185E38093A50124E230E002C024E262
:100AF00035E8C901089565E971E082E991E00E9455
:100B00007E08E6CF6F927F928F929F92BF92CF9294
:100B1000DF92EF92FF920F931F93DF93CF9300D05A
:100B2000CDB7DEB782E08093E9008091E80082FFD4
:100B3000D2C2189A982F9B7F9093E800E2E6F1E0EA
:100B40008091F100819321E0E138F207C9F79F77A6
:100B50009093E8008091620190916301A0916401FB
:100B6000B091650185559345A244B34489F48091C1
:100B70006F01882369F420916E01822F90E08F71BC
:100B80009070892B29F4809170018150803148F058
:100B900091E29093EB0081E08093E9009093EB0069
:100BA00086C280916A0190916B01A0916C01B09115
:100BB0006D0181509240A040B040C8F427FF0FC0A3
:100BC00081E08093E90040916A0150916B0122E835
:100BD00031E0C90160E070E00E94850808C06091C2
:100BE0006A0170916B0182E891E00E94FB0485E547
:100BF00093E5A2E4B3E58093840390938503A093E7
:100C00008603B09387038091660190916701A0915C
:100C10006801B09169018093880390938903A09340
:100C20008A03B0938B0310928C0310928D03109261
:100C30008E0310928F0390916F0183E1989FF001D2
:100C40001124E050FF4F2F0120917101722F7F730B
:100C50007A837D3109F439C27E31B0F4723109F4FE
:100C600056C0733138F47130B1F1713068F17330BE
:100C700041F53AC08A818A3109F44CC08B3109F4BC
:100C8000AEC08531F1F421C2AA81A83209F428C18D
:100C9000A93248F4A33209F4B7C0A53209F4E9C077
:100CA000AE3179F4A9C0BA81BB3209F48AC1BC3231
:100CB00018F4BA3231F414C18A818E52823008F4A9
:100CC0000FC100E215E8AEC18481882309F0FDC19F
:100CD0000AE312E8A3C10E94E9038C01009709F01E
:100CE0008BC10E94950387C180E780938201F20146
:100CF0008089809384018AE080938901818980932F
:100D00008E01828980938F0102E110E077C10E94F9
:100D1000220571C1909173019F7384E980938401CE
:100D200080E8809385019B31F1F09C3128F491306B
:100D300051F0953029F411C09C3111F19F3359F1D4
:100D4000EAE8F1E043C090938A018AE080938B0146
:100D500010928C01E5E9F1E039C08AE891E00E9447
:100D60004B03FC0133C090938A018AE080938B018E
:100D700010928C0181E080938D01E6E9F1E026C0BC
:100D800090938A0186E080938B0185E080938D01AA
:100D9000E2E9F1E01BC001E000938A011AE0109340
:100DA0008B0110928C0185E991E00E944B03DC01DC
:100DB000FC018BE1819311961C93118202838CE1DB
:100DC000838786E0848785E08687739682E891E052
:100DD0008E2E881A80928301082D10E00FC1809119
:100DE000750181FD0EC080FF03C00E94E90303C1AD
:100DF00087810E945F0469C180917501882309F48D
:100E000064C104E215E80AC180898823A9F588E055
:100E100080938501F201348525859685408551852D
:100E20008481882311F460E001C062E0239F900177
:100E30001124892F90E0DC012A9FC0012B9F900D87
:100E40003A9F900D11240197292F332727FD3A95BA
:100E5000209388018093890160938A01852F9927C7
:100E600087FD9A9580938C0140938D010CE010E0F2
:100E7000C5C08089882319F00FEF1FEFCFC0848190
:100E8000882331F40E94E9038C01009709F0B4C073
:100E9000F2014085518525858485289F9001112484
:100EA000868590E0FC012E9FC0012F9F900D3E9FF4
:100EB000900D11240197292F332727FD3A95209370
:100EC00084018093850110928601852F992787FDE3
:100ED0009A95809388014093890108E010E08EC0C4
:100EE000809179019091780127FF03C0982F80911C
:100EF0007A017C01009709F4E8C00E94E9038C01A3
:100F0000009709F079C0FA81FB71F983FA3009F092
:100F1000D0C01C99CEC0DCC00894611C711CF201C9
:100F20008485660C771C781610F0781A6394BA944E
:100F3000C1F7962D858581FF0AC0862D90E060FE61
:100F400002C02E9801C02E9A95958795982F892FCB
:100F50000E94B2038C01009709F04EC029812A300B
:100F600031F482E891E060E072E00E94FB045D9859
:100F700088EC90E0F6013197F1F70197D9F7872DCA
:100F80008F5F0E947B085D9A3981383031F482E8A6
:100F900091E060E072E00E94D4040894E108F10856
:100FA000E114F10409F0B8CF84E1D20116968C93D4
:100FB00010926A0110926B0110926C0110926D01F7
:100FC0001DC00E94E9038C010097B1F48091760165
:100FD00090917501F20125854485249F900111248B
:100FE00048E0880F991F921710F0921B83954A953D
:100FF000C1F70E94B2038C0117FD10C080916A01F5
:1010000090916B01A0916C01B0916D018150924063
:10101000A040B040A4F000E812E804C0FFEF0F3F8A
:101020001F0729F0F201C8019F70908B818B81E02E
:101030008093E90081E28093EB0081E016C060912B
:101040006A0170916B01C801861B970B97FD04C064
:1010500090938D0380938C0382E891E00E94D404E6
:10106000F201108A118A128A80E08093900311E0C5
:101070000E94BF011093E9008091EB0085FDF8CF3D
:101080008091E80080FFFCCF8091E8008E7F809304
:10109000E800E4E8F3E081918093F10023E0E13996
:1010A000F207C9F78091E8008F778093E800189ADB
:1010B00012C080917601909175013C0138E0B32E09
:1010C00020E9C22E21E0D22E2ACF00E010E096CFF8
:1010D00007E217E8A3CF0F900F90CF91DF911F91F8
:1010E0000F91FF90EF90DF90CF90BF909F908F90E7
:1010F0007F906F90089582E193E80895FB01DC01F1
:1011000005900D920020E1F70895DC0101C06D9378
:0C11100041505040E0F70895F894FFCFE4
:10111C0005010250000000010002F4010F02500111
:10112C0000000000000000000000000000000000B3
:10113C0000000000000000000000000000000000A3
:10114C000000000000000000000000000000000093
:10115C000000000000000000000000000000000083
:10116C000000000000000000000000000000000073
:00000001FF
